:020000040000FA
:100000000C94C5010C94ED010C94ED010C943B167D
:100010000C943B160C943B160C94ED010C94ED01E2
:100020000C94ED010C94ED010C94ED010C94ED0198
:100030000C94ED010C94ED010C94ED010C94ED0188
:100040000C94F1150C94ED010C94BF150C949915BA
:100050000C94ED010C94ED010C94ED010C94ED0168
:100060000C94B3160C94ED0107634236B79BD8A7E6
:100070001A39685618AEBAAB558C1D3CB7CC5763CD
:10008000BD6DEDFD753EF6177231BF000000803F7B
:1000900008000000BE922449123EABAAAA2ABECD97
:1000A000CCCC4C3E00000080BEABAAAAAA3E000009
:1000B0000000BF000000803F000000000008417801
:1000C000D3BB4387D1133D190E3CC3BD4282AD2B38
:1000D0003E68EC8276BED98FE1A93E4C80EFFFBE30
:1000E00001C4FF7F3F00000000004E414E494E49D1
:1000F0005459494E46CDCCCC3D0AD7233C17B7D1F5
:100100003877CC2B329595E6241FB14F0A0000209A
:10011000410000C84200401C4620BCBE4CCA1B0E19
:100120005AAEC59D7400407A10F35A00A0724E1862
:10013000090010A5D4E80000E87648170000E40B99
:1001400054020000CA9A3B000000E1F5050000805F
:10015000969800000040420F000000A086010000B9
:1001600000102700000000E8030000000064000009
:100170000000000A00000000000100000000002C48
:1001800076D888DC674F0823DFC1DFAE59E1B1B70D
:1001900096E5E3E453C63AE651997696E8E6C284DA
:1001A00026EB898C9B62ED407C6FFCEFBC9C9F40F2
:1001B000F2BAA56FA5F490055A2AF75C936B6CF917
:1001C000676DC11BFCE0E40D47FEF520E6B500D0ED
:1001D000ED902E0300943577050080841E08000002
:1001E000204E0A000000C80C333333330F986E12D0
:1001F000831141EF8D2114893BE65516CFFEE6DBD6
:1002000018D1844B381BF77C1D901DA4BBE424201F
:100210003284725E228100C9F124ECA1E53D2754AD
:100220003D0020572F6D5E3220555620496E746573
:100230006E7369747900234E6F20504D2073656E84
:10024000736F722100504D28312E302C322E352CF8
:100250003130293D00206C78204C69676874204952
:100260006E74656E7369747900495220466C616DD5
:1002700065204C6576656C3D00476173206C657642
:10028000656C3D0023496E76616C6964206B65790D
:10029000210000000000240027002A0023626D7066
:1002A000206661696C6564002357656C636F6D65DA
:1002B00020746F20757365204E616E6F204C6F67E0
:1002C000676572004D533D00235556207A65726F65
:1002D00020766F6C74616765203D00503D0042548C
:1002E0003D004448543D00234475726174696F6E4B
:1002F0003D0054494D45443D0023496E7465727676
:10030000616C3D0054494D45493D0053484F57539A
:100310003D004C6F67676572204E616D653A200045
:100320004C4F474745520056455253494F4E005295
:1003300045424F4F54000000000800020100000336
:10034000040700000000000000000000000023007F
:100350002600290000000000250028002B000404CE
:10036000040404040404020202020202030303035D
:100370000303010204081020408001020408102039
:10038000010204081020D217392011241FBECFEF1C
:10039000D8E0DEBFCDBF11E0A0E0B1E0E0E1FAE5DA
:1003A00002C005900D92A83DB107D9F724E0A8ED51
:1003B000B1E001C01D92AB36B207E1F711E0C4EC29
:1003C000D1E004C02197FE010E94DE2AC33CD10780
:1003D000C9F70E9434190C94FB2C0C94000008956A
:1003E00008950895AF92BF92CF92DF92EF92FF925D
:1003F0000F931F93CF93DF936C017B018B01040F4D
:10040000151FEB015E01AE18BF08C017D10759F0E8
:100410006991D601ED91FC910190F081E02DC6012A
:100420000995892B79F7C501DF91CF911F910F9124
:10043000FF90EF90DF90CF90BF90AF900895CF9353
:10044000DF93FC0144815581608171818BEE92E0E4
:100450000E94F201EC0142E050E06AE471E08BEEB0
:1004600092E00E94F2018C0F9D1FDF91CF910895C1
:10047000FC01538D448D252F30E0842F90E0821BAA
:10048000930B541710F0CF96089501970895FC012F
:10049000918D828D981761F0A28DAE0FBF2FB11D87
:1004A0005D968C91928D9F5F9F73928F90E00895DF
:1004B0008FEF9FEF0895FC01918D828D981731F099
:1004C000828DE80FF11D858D90E008958FEF9FEFED
:1004D0000895FC01918D228D892F90E0805C9F4FC3
:1004E000821B91098F73992708958BEE92E00E94E9
:1004F000690221E0892B09F420E0822F089580E031
:1005000090E0892B29F00E94750281110C94000063
:100510000895FC01A48DA80FB92FB11DA35ABF4F98
:100520002C91848D90E001968F739927848FA689F2
:10053000B7892C93A089B1898C91837080648C9346
:10054000938D848D981306C00288F389E02D8081F5
:100550008F7D80830895EF92FF920F931F93CF9327
:10056000DF93EC0181E0888F9B8D8C8D98131AC0EE
:10057000E889F989808185FF15C09FB7F894EE89D5
:10058000FF896083E889F989808183708064808332
:100590009FBF81E090E0DF91CF911F910F91FF907D
:1005A000EF900895F62E0B8D10E00F5F1F4F0F7325
:1005B0001127E02E8C8D8E110CC00FB607FCFACFE0
:1005C000E889F989808185FFF5CFCE010E948902F3
:1005D000F1CFEB8DEC0FFD2FF11DE35AFF4FF082B1
:1005E0009FB7F8940B8FEA89FB8980818062CFCF17
:1005F000CF93DF93EC01888D8823B9F0AA89BB895A
:10060000E889F9898C9185FD03C0808186FD0DC044
:100610000FB607FCF7CF8C9185FFF2CF808185FF65
:10062000EDCFCE010E948902E9CFDF91CF910895ED
:10063000833081F028F4813099F08230A9F0089558
:100640008730A9F08830C9F08430B1F480918000FF
:100650008F7D03C0809180008F7780938000089504
:1006600084B58F7784BD089584B58F7DFBCF80914D
:10067000B0008F778093B00008958091B0008F7D97
:10068000F9CFCF93DF93E5E4F3E08491E1E8F3E081
:10069000D491EDE6F3E0C491CC23A1F081110E9446
:1006A0001803EC2FF0E0EE0FFF1FE65BFC4FA59167
:1006B000B491EC91ED2381E090E009F480E0DF91CA
:1006C000CF91089580E090E0FACF1F93CF93DF930E
:1006D000282F30E0F901EA5CFC4F8491F901EE58D3
:1006E000FC4FD491F901E25AFC4FC491CC23A9F0FC
:1006F000162F81110E941803EC2FF0E0EE0FFF1F60
:10070000EC5AFC4FA591B4918FB7F894EC9111116C
:1007100008C0D095DE23DC938FBFDF91CF911F916E
:100720000895DE2BF8CFCF93DF9390E0FC01EE58D5
:10073000FC4F2491825A9C4FFC0184918823D1F074
:1007400090E0880F991FFC01EE56FD4FA591B491E2
:10075000FC01EC5AFC4FC591D49161110EC09FB7BA
:10076000F8948C91E22FE0958E238C932881E223DC
:10077000E8839FBFDF91CF9108958FB7F894EC91F4
:10078000E22BEC938FBFF6CF8E3008F08E50209185
:10079000000190E4299F900111248770822B80939F
:1007A0007C0080917A00806480937A0080917A0046
:1007B00086FDFCCF809178009091790008953FB735
:1007C000F8948091650290916602A0916702B091C1
:1007D000680226B5A89B05C02F3F19F00196A11D00
:1007E000B11D3FBFBA2FA92F982F8827BC01CD017B
:1007F000620F711D811D911D42E0660F771F881FDA
:10080000991F4A95D1F708958F929F92AF92BF9208
:10081000CF92DF92EF92FF926B017C010E94DF0387
:100820004B015C01C114D104E104F104B9F00E9450
:10083000DF03681979098A099B09683E73408105BD
:10084000910580F321E0C21AD108E108F10888EE91
:10085000880E83E0981EA11CB11CE4CFFF90EF909E
:10086000DF90CF90BF90AF909F908F9008958F9220
:100870009F92AF92BF92EF92FF921F93CF93DF931D
:10088000C82F10925F0410926004109261041092BD
:1008900062041092630461E08FE00E94930360E0C1
:1008A0008FE00E9465036C2F70E090E080E00E9472
:1008B000040460E08FE00E9493038BE990E00197CD
:1008C000F1F7C0E9D1E00E944103892B71F421972F
:1008D000D1F78EEF9FEFDF91CF911F91FF90EF90B7
:1008E000BF90AF909F908F900895C0E9D1E00E9493
:1008F0004103019719F42197D1F7EBCFD8E2C0E873
:1009000010E090E9E92EFF24F3940E944103892B23
:1009100029F481E0E81AF108C1F7DBCF0E94DF0378
:100920004B015C0180E9E82EFF24F3940E9441030F
:10093000019729F481E0E81AF108C1F7CACF0E94B3
:10094000DF03681979098A099B09693271058105F4
:10095000910538F0E12FF0E0E95AFB4F80858C2BB0
:100960008087C69511F41F5FC0E8D15051F690E022
:1009700080E0B1CF8F929F92AF92BF92CF92DF92E1
:10098000EF92FF920F931F93CF93DF938AE0A82EED
:10099000B12CD0E0C0E0EE24EA9493E0F92E882454
:1009A0008A9423E0922ED12CC12C10E000E08FE03D
:1009B0000E94C4030817190790F1C816D90608F455
:1009C0006C018815990568F18E159F0508F47C0166
:1009D000C80FD91F65E070E080E090E00E94040439
:1009E00081E0A81AB10819F70C0D1D1DCE01801B5E
:1009F000910B8E199F098819990966E070E00E9491
:100A00006A29CB01DF91CF911F910F91FF90EF9059
:100A1000DF90CF90BF90AF909F908F9008958C0102
:100A2000D0CF4C01D5CF2FB7F8946091610270916F
:100A3000620280916302909164022FBF0895209119
:100A40005E0230915F022817390771F490915D02C0
:100A500080915C02981741F0E0915D02F0E0E45E65
:100A6000FD4F808190E008958FEF9FEF08950895E6
:100A7000EF92FF920F931F93CF93DF93DC015C966D
:100A8000ED90FC905D97E114F10479F481E090E041
:100A900013969C938E93129790E080E0DF91CF9114
:100AA0001F910F91FF90EF9008955196ED91FC9159
:100AB000529750968C915097982F90950FB75E96BD
:100AC0002C915E97122F127021FD6095F894208171
:100AD000112319F1282B2083E7012197F1F728E052
:100AE000462F50E0308160FF1AC0382B3083E70179
:100AF0002197F1F7BA0175956795215089F7112370
:100B000081F08081892380830FBF5C968D919C91B9
:100B10000197F1F781E090E0C1CF2923DCCF3923A1
:100B2000E5CF9081892BEFCF20915E0230915F025B
:100B30002817390771F480915C0220915D0290E0E2
:100B4000805C9F4F821B910960E470E00E947E29C7
:100B5000089590E080E0089520915E0230915F0258
:100B600028173907B9F490915D0280915C029817BB
:100B700089F0E0915D02F0E0E45EFD4F808120911C
:100B80005D0230E02F5F3F4F2F73332720935D02CC
:100B900090E008958FEF9FEF08950F931F930E94A9
:100BA0001305609340047093410480934204909332
:100BB000430488E394E00E94AC0597FF1DC00E94A7
:100BC000130500914004109141042091420430919A
:100BD0004304601B710B820B930B00913C0410913A
:100BE0003D0420913E0430913F0460177107820755
:100BF0009307F8F28FEF9FEF1F910F910895E09107
:100C00005E02F0915F02E817F90769F4A389B489DD
:100C10009C918589809589238C9310925F02109214
:100C20005E0281E0089580E008952091F901260F89
:100C30003327331F21323105ECF42091C102FC012E
:100C400090E080E0243069F082E00895A091F901FD
:100C50002191AC0147525E4FA40FB52FB11D2C93CB
:100C60000196861798F38091F901680F6093F90156
:100C700080E0089581E008951092C10281E08093A0
:100C8000C00210929B0261E082E10E94650361E074
:100C900083E10E946503E9EBF0E080818E7F808331
:100CA00080818D7F808388E48093B80085E4809381
:100CB000BC00089510927A02109279021092C80234
:100CC0001092EA020E943C068FEE91E09093780227
:100CD0008093770280EF91E0909376028093750283
:100CE0000895CF93DF9391E09093D8018823B9F0D2
:100CF000C091B800D091BA008091BC008A7B8093EB
:100D0000BC0060E082E10E94650360E083E10E9434
:100D100065030E943C06D093BA00C093B800DF91EF
:100D2000CF910895CF92DF92EF92FF920F931F938E
:100D3000CF93DF93D091EA0281E0D13208F09CC0DA
:100D4000C091E9020E94DF036B017C018091C10226
:100D500081116CC082E08093C10281E08093C00267
:100D60008FEF8093BF021092BE02D093BD02A9EC18
:100D7000B2E0EDE9F2E080E0D8138DC010929C0261
:100D800080919C02CC0FC82BC0939C0280919B0247
:100D9000813009F084C010929B020E94DF036B0136
:100DA0007C0180919C028093BB008091C302909152
:100DB000C402A091C502B091C602892B8A2B8B2B4D
:100DC000A1F00E94DF030091C3021091C4022091A0
:100DD000C5023091C6026C197D098E099F0906175C
:100DE00017072807390708F442C08091BC0083FD2B
:100DF000D8CF85EC8093BC000E94DF036B017C019F
:100E00008091C102823009F44CC08091BF028F3FB3
:100E100009F469C08091BF02803209F466C08091F4
:100E2000BF02803309F463C084E026C08091C3020E
:100E30009091C402A091C502B091C602892B8A2B61
:100E40008B2B09F483CF0E94DF030091C302109122
:100E5000C4022091C5023091C6026C197D098E0929
:100E60009F09061717072807390708F06FCF8091E9
:100E7000C2020E94710685E01092C8021092EA0236
:100E80001092C702DF91CF911F910F91FF90EF90C9
:100E9000DF90CF9008959D9191938F5F6DCF85EEF8
:100EA000A9CF8091C3029091C402A091C502B091D4
:100EB000C602892B8A2B8B2B09F4A2CF0E94DF0359
:100EC0000091C3021091C4022091C5023091C60264
:100ED0006C197D098E099F0906171707280739071E
:100EE00008F08ECFC4CF80E0C7CF82E0C5CF83E0CB
:100EF000C3CFCF92DF92EF92FF920F931F93CF93C6
:100F0000DF93D82FC62F613208F098C00E94DF030C
:100F10006B017C018091C10281116BC081E08093E3
:100F2000C1028093C0029FEF9093BF021092BE0255
:100F30009C0F9093BD0280939C0280919C02DD0FD8
:100F4000D82BD0939C0280919B02813009F078C00D
:100F500010929B020E94DF036B017C0180919C0236
:100F60008093BB008091C3029091C402A091C502FE
:100F7000B091C602892B8A2B8B2BA1F00E94DF0334
:100F80000091C3021091C4022091C5023091C602A3
:100F90006C197D098E099F0906171707280739075D
:100FA00008F448C08091BC0083FDD8CF85EC8093C5
:100FB000BC000E94DF036B017C018091C102813083
:100FC00009F440C08091BE028C1710F4C091BE029B
:100FD000EDE9F2E0ABE7B2E080E08C1355C08C2F76
:100FE000DF91CF911F910F91FF90EF90DF90CF9005
:100FF00008958091C3029091C402A091C502B0915E
:10100000C602892B8A2B8B2B09F484CF0E94DF0325
:101010000091C3021091C4022091C5023091C60212
:101020006C197D098E099F090617170728073907CC
:1010300008F070CF8091C2020E947106C0E0CFCF4D
:1010400085EEB5CF8091C3029091C402A091C502F4
:10105000B091C602892B8A2B8B2B09F4AECF0E944C
:10106000DF030091C3021091C4022091C5023091A8
:10107000C6026C197D098E099F09061717072807F4
:10108000390708F09ACFD6CF91919D938F5FA5CF66
:10109000E0917A0280917902E81730F4F0E0E558A7
:1010A000FD4F808190E008958FEF9FEF089590911C
:1010B0007A02809179022FEF3FEF981748F4E92FD9
:1010C000F0E0E558FD4F208130E09F5F90937A0279
:1010D000C90108958091790290917A02891B990B38
:1010E0000895CF92DF92EF92FF920F931F93CF93C9
:1010F000DF937C01CB018A012091C702222389F072
:10110000EB016B01C40ED51ECC15DD0569F06991AC
:10111000D701ED91FC910190F081E02DC701099577
:10112000F3CF642F0E941506C801DF91CF911F9164
:101130000F91FF90EF90DF90CF900895CF93DF93C2
:101140001F92CDB7DEB769832091C7022223F9F041
:101150002091EA02203258F021E030E0FC01338394
:10116000228390E080E00F90DF91CF9108958091ED
:10117000C802E82FF0E0E753FD4F998190838F5F1D
:101180008093C8028093EA0281E090E0ECCF61E0B6
:10119000CE0101960E941506F7CF90E080E00895F9
:1011A0008F929F92AF92BF92CF92DF92EF92FF9277
:1011B000CF93DF93CAE0D4E0988121E02093C70267
:1011C0009093E9021092C8021092EA02682F88E810
:1011D00093E00E949E080E94920663E088810E942C
:1011E000790710927A028093790288E893E00E944E
:1011F0005708092E000CAA0BBB0B8824982EA92E89
:10120000BA2E88E893E00E945708092E000CAA0B1A
:10121000BB0B6C017D01C828D928EA28FB28FE2CCD
:10122000ED2CDC2CCC2488E893E00E945708BC010C
:10123000990F880B990B6C297D298E299F29DF91A5
:10124000CF91FF90EF90DF90CF90BF90AF909F90A5
:101250008F9008958F929F92AF92BF92CF92DF921C
:10126000EF92FF920F931F93209113042F3F19F4D5
:101270008AEF0E94D008009117041091180430E002
:1012800020E0C72ED82EE92EFF24E7FCFA94C01ADE
:10129000D10AE20AF30A57E0959587957795679505
:1012A0005A95D1F7000F111F221F331F4B015C010C
:1012B000801A910AA20AB30AA5019401A091190407
:1012C000B0911A040E94F2254B015C01FBE0B59439
:1012D000A79497948794FA95D1F7A7019601C7012F
:1012E000B6010E945A299B01AC01ACE05595479587
:1012F00037952795AA95D1F7A0911B04B0911C04AE
:101300000E94F2259B01AC01BEE0559547953795AB
:101310002795BA95D1F7280D391D4A1D5B1D2093DD
:101320000F04309310044093110450931204A5E06D
:10133000B0E00E94E72560587F4F8F4F9F4F672F87
:10134000782F892F992787FD9A950E94B12420E054
:1013500030E048EC52E40E94CF261F910F91FF909D
:10136000EF90DF90CF90BF90AF909F908F900895B7
:101370002F923F924F925F926F927F928F929F92A5
:10138000AF92BF92CF92DF92EF92FF920F931F9393
:10139000CF93DF93CDB7DEB76B970FB6F894DEBF70
:1013A0000FBECDBF0E942A09809113048F3F39F4EC
:1013B00087EF0E94D0086E8B7F8B888F998F8091EA
:1013C0000F0490911004A0911104B09112046C01CB
:1013D0007D01FF0CCC08DC2C76019C01AD016C2D4D
:1013E0007C2D8C2D9C2D345F414051096109710980
:1013F0008109910929873A874B87652E762E872E9A
:10140000982E9B8F5901C42ED52EE62EF72E082F2D
:10141000192F0E949229322E232E488B598B6A8BCA
:101420007B8B8C8B9D8B3091200420911F04932FFC
:10143000990F990B492F592F692F792F892F0E94C6
:1014400092290CE00E948A2A29833C874A8F5D8773
:101450006E877F87582E492E3091220420912104D7
:10146000932F990F990BA32CB22CC888D988EA889E
:10147000FB880C891D89492F592F692F792F892FB6
:101480000E94922908E00E94A32AA980BC84CA8CE9
:10149000DD84EE84FF84052D142D0E94C02A70582F
:1014A0008F4F9F4FE0911D04F0911E045F01D12CDE
:1014B000C12CE12CF12C8701E983BA82CB82DC823A
:1014C000ED82FE820F831887C12CD12CE12CF12CE8
:1014D00000E010E00E94922901E20E94A32A2A8FD4
:1014E000532E49835C876D877E878F87492EA0E0C6
:1014F0000E94D22A09F436C1309128042091270491
:10150000932F990F990BA32CB22CC888D988EA88FD
:10151000FB880C891D89492F592F692F792F892F15
:101520000E9492291901488B598B6A8B7B8B8C8B7B
:101530009D8B3091260420912504932F990F990BB0
:10154000A984BA84CB84D62CE72CF82C092D1B8DCA
:10155000492F592F692F792F892F0E94922901E154
:101560000E948A2A5101C888D988EA88FB880C8998
:101570001D890E94C02A59016A017B01382E192F4A
:101580004E895F89688D798D84E07595679557954B
:1015900047958A95D1F780E090E0A0E1B0E0841B08
:1015A000950BA60BB70B3C014D01990C6608762CE8
:1015B00043019C01AD01662D762D862D962D0FE100
:1015C0000E948A2A722E832E942E5987B62FA72F17
:1015D000F82FE92F3091240420912304932F990FA1
:1015E000990B492F592F692F792F892F03E20E94D8
:1015F0008A2A032D0E94C02A59016A017B018C01AD
:10160000272D382D492D59856B2F7A2F8F2F9E2FFF
:101610000E94C92AE5E3AE2EFCE0BF2EC12CD12CDE
:10162000E12CF12C00E010E00E949229AA8CB52C4C
:10163000C980DC84ED84FE840F85142D0E94EC2982
:101640002F873E8749875A876B8779838C879D8749
:101650000DE00E94A32A922E832E742E652E562E04
:10166000472E382E292E30912E0420912D04932FB1
:10167000990F990BA92CB82CC72CD62CE52CF42C3F
:10168000032D122D492F592F692F792F892F0E9451
:1016900092290E94922909E10E94A32AAF84BE8464
:1016A000C984DA84EB84F9800C851D850E94C02AE8
:1016B00019012A013B014C0130912C0420912B048B
:1016C000932F990F990B492F592F692F792F892F14
:1016D0000E94922903E10E94A32A59016A017B0119
:1016E0008C019101A201B301C4010E94C02A08E04B
:1016F0000E94A32A59016A017B01E82F192F30911A
:101700002A0420912904932F990F990B492F592FBF
:10171000692F792F892F04E00E948A2A0E2F0E94B8
:10172000C02A0E94772720E030E040E85BE30E9477
:1017300010256B960FB6F894DEBF0FBECDBFDF91BC
:10174000CF911F910F91FF90EF90DF90CF90BF90BE
:10175000AF909F908F907F906F905F904F903F9051
:101760002F90089560E070E0CB01E3CFCF9390918C
:1017700013049F3F41F5682F80910A0491E09093F4
:10178000C7028093E9021092C8021092EA0288E828
:1017900093E00E949E080E94920662E080910A04F3
:1017A0000E94790710927A028093790288E893E088
:1017B0000E945708C82F88E893E00E94570820E04D
:1017C0003C2F282B392B922F832FCF910895AF9246
:1017D000BF92DF92EF92FF920F931F93CF93DF930D
:1017E0005C0104E913E0D0E0C0E0F801D1908F0182
:1017F0007501EC0EFD1EC7010E94D125D81621F0FF
:101800006D2DC7010E94D9252196CC34D10569F7E9
:1018100084E993E0DF91CF911F910F91FF90EF90BA
:10182000DF90BF90AF90089585ED8093BC008091CC
:10183000C3029091C402A091C502B091C60207965E
:10184000A11DB11D23E0B695A795979587952A957B
:10185000D1F72091BC0024FD03C01092C10208956D
:101860004091C3025091C4026091C5027091C602BA
:10187000452B462B472B69F30097A105B10541F095
:1018800025E32A95F1F700000197A109B109E1CFFD
:101890008091C2020C947106FC01808191810097B5
:1018A00011F00C94812060E070E0CB010895FB0101
:1018B00044815581FC01248135812417350778F056
:1018C00080819181009759F0FB01608171816115E0
:1018D000710529F00E94DE2C21E0892B09F020E01F
:1018E000822F08950F931F93CF93DF938C01EB0109
:1018F000FC01808191810097E1F068817981611517
:101900007105A9F0428153812C813D814217530713
:1019100070F00E94D72C8C819D81F801958384837F
:101920001D821C82DF91CF911F910F9108950E941B
:10193000802B88819981F801918380838A819B81A2
:10194000938382838C819D819583848319821882FD
:101950001B821A82E5CFCF93DF93EC0188819981B6
:10196000009711F00E94802B198218821D821C8220
:101970001B821A82DF91CF910895FC0180819181B1
:10198000009711F00C94802B08950F931F93CF9321
:10199000DF93EC0188819981009759F02A813B817E
:1019A0002617370730F081E0DF91CF911F910F911B
:1019B00008958B016F5F7F4F0E94092C009759F0AB
:1019C000998388831B830A832C813D81232B59F7BC
:1019D000FC011082E8CF80E0E7CFEF92FF920F93F7
:1019E0001F93CF93DF936115710541F480E0DF9180
:1019F000CF911F910F91FF90EF90089541155105E0
:101A0000B1F07B01EC010C811D81040F151FB801A1
:101A10000E94C50C882351F3288139818C819D81D6
:101A2000B701820F931F0E94D72C1D830C8381E086
:101A3000DECFFC01448155816081718184E094E0B6
:101A40000C94ED0CCF93DF93EC01FB01019000208F
:101A5000E9F73197AF01461B570B0E94ED0C81113E
:101A600003C0CE010E94AB0CCE01DF91CF9108954F
:101A7000CF93DF93EC01FB0144815581608171813B
:101A80000E94ED0C811103C0CE010E94AB0CCE016F
:101A9000DF91CF910895EF92FF920F931F93CF9311
:101AA000DF93EC018B01CB010E94AF207C01BC01D4
:101AB000CE010E94C50C81110BC0CE010E94AB0C5F
:101AC000CE01DF91CF911F910F91FF90EF9008957C
:101AD000FD82EC82B801888199810E94A820F0CF14
:101AE000FC011182108213821282158214820C94DE
:101AF0004B0DEF92FF920F931F93CF93DF93EC0167
:101B00007B018A01BA010E94C50C81110BC0CE0174
:101B10000E94AB0CCE01DF91CF911F910F91FF90EE
:101B2000EF9008951D830C83B701888199810E94ED
:101B3000D72CF0CFFB0101900020E9F73197AF01DE
:101B4000461B570B0C94790D0F931F93CF93DF9384
:101B5000CDB7DEB762970FB6F894DEBF0FBECDBF2C
:101B60008C01CB01F801118210821382128215823E
:101B700014824AE0BE016F5F7F4F0E94B820BE0111
:101B80006F5F7F4FC8010E949A0D62960FB6F8945E
:101B9000DEBF0FBECDBFDF91CF911F910F91089592
:101BA000CF93DF93EC01FB018617970749F0608123
:101BB00071816115710541F0448155810E94790D53
:101BC000CE01DF91CF9108950E94AB0CF9CFFC01BB
:101BD0001182108213821282158214820C94D00D0D
:101BE000FC01118210821382128215821482FB0181
:101BF00001900020E9F73197AF01461B570B0C9479
:101C0000790DAF92BF92CF92DF92EF92FF920F9336
:101C10001F93CF93DF936C015B017A018901241735
:101C2000350720F48F2D7901042F182F6CE471E013
:101C3000C6010E94F00DD5011496CD91DC91EC16F1
:101C4000FD06E0F40C171D0708F4E801D501ED913D
:101C5000FC911197EC0FFD1F108110826D917C910A
:101C60006E0D7F1DC60161157105A1F00E949A0DD0
:101C7000F50180819181C80FD91F1883C601DF91BA
:101C8000CF911F910F91FF90EF90DF90CF90BF9079
:101C9000AF9008950E94AB0CEBCF0F931F93CF939F
:101CA000DF93CDB7DEB72C970FB6F894DEBF0FBE2B
:101CB000CDBFFC01248135811216130664F48C011A
:101CC000253131059CF40E941F026FE070E080E036
:101CD00090E00E9404042C960FB6F894DEBF0FBE6D
:101CE000CDBFDF91CF911F910F9108952FE030E08C
:101CF00050E040E0BC01CE0107960E94010E4B85EA
:101D00005C856F8178858BEE92E00E94F20169E13B
:101D100070E080E090E00E940404F80124813581A5
:101D20004FE050E0B801CE0101960E94010EBE01C5
:101D30006F5F7F4FCE0107960E94720CCE01019615
:101D40000E94BD0CCE0107960E941F026FE070E05A
:101D500080E090E00E9404046CE471E0CE010796FC
:101D60000E949A0DCE0107960E94BD0CB4CFEF924F
:101D7000FF920F931F93CF93DF93CDB7DEB7A19759
:101D80000FB6F894DEBF0FBECDBF7C01CB01BA0108
:101D9000F70111821082138212821582148242E0AE
:101DA000420F8E010F5F1F4F0E945F20009789F046
:101DB000BC01C7010E949A0DA1960FB6F894DEBF30
:101DC0000FBECDBFDF91CF911F910F91FF90EF908C
:101DD0000895C7010E94AB0CEFCF8F929F92AF92F4
:101DE000BF92EF92FF920F931F93CF93DF93CDB7E4
:101DF000DEB72C970FB6F894DEBF0FBECDBF64E6FA
:101E000070E080E090E00E940404809104019091D1
:101E100005010B9731F580916404882309F0F8944B
:101E200082E10E9437048C0180916404882309F0C8
:101E300078940115110509F4BAC080E090ECA9E787
:101E4000B4EC8093570490935804A0935904B09332
:101E50005A0480935B0490935C04A0935D04B09358
:101E60005E048091040190910501469731F58091BF
:101E70006404882309F0F89481E00E9437048C01FF
:101E800080916404882309F078940115110509F400
:101E9000EFC080E090ECA9E7B4EC809357049093F6
:101EA0005804A0935904B0935A0480935B04909310
:101EB0005C04A0935D04B0935E0464E670E080E08F
:101EC00090E00E940404012B09F060C040915B0483
:101ED00050915C0460915D0470915E0421E0CE013C
:101EE00007960E94B70E6DE471E0CE0101960E9444
:101EF000F00DBE01695F7F4FCE0101960E94380D43
:101F000060E571E00E94220DBC0184E094E00E9433
:101F1000D00DCE0101960E94BD0C40915704509106
:101F200058046091590470915A0421E0CE01019641
:101F30000E94B70EBE016F5F7F4FCE0107960E94D1
:101F4000720CCE0101960E94BD0C64E571E0CE01D9
:101F500001960E94F00DBE01695F7F4FCE01019690
:101F60000E94380D67E571E00E94220D0E94190D54
:101F7000CE0101960E94BD0C64E670E080E090E026
:101F80000E940404CE0107960E94BD0C2C960FB649
:101F9000F894DEBF0FBECDBFDF91CF911F910F919F
:101FA000FF90EF90BF90AF909F908F900895109109
:101FB0005F04E09060046E2D70E090E080E00E948D
:101FC000B1242DEC3CEC4CEC5DE30E9410254B0160
:101FD0005C01612F70E090E080E00E94B1249B01E1
:101FE000AC01C501B4010E9463266093570470934D
:101FF00058048093590490935A0400916104F0901E
:102000006204602F6F7770E090E080E00E94B1245E
:102010004B015C016F2D70E090E080E00E94B124E4
:102020002DEC3CEC4CEC5DE30E9410259B01AC01D7
:10203000C501B4010E94632607FD18C060935B04CC
:1020400070935C0480935D0490935E041E0D100FEA
:102050001F0D81E090E020916304121302C090E014
:1020600080E000271127081B190BFBCE9058E6CF04
:102070001091600400915F0460915F0470916004AE
:1020800076276727762790E080E00E94AF242DEC2A
:102090003CEC4CEC5DE30E94102560935704709378
:1020A00058048093590490935A04E0906204F0908D
:1020B00061046F2D6F77762F6E2D90E080E00E9487
:1020C000AF242DEC3CEC4CEC5DE30E941025F7FCBA
:1020D00018C060935B0470935C0480935D049093DC
:1020E0005E04100F1E0D1F0D81E090E0209163042F
:1020F000121302C090E080E000271127081B190B83
:10210000DCCE9058E6CF4F925F926F927F928F9283
:102110009F92AF92BF92CF92DF92EF92FF92CF93B6
:10212000DF93CDB7DEB72C970FB6F894DEBF0FBEA6
:10213000CDBF0E94B8092B013C010E942A094B0126
:102140005C016091A0037091A1038091A203909122
:10215000A3030E94B12420E030E048EC52E40E9446
:10216000CF266B017C010E94B80920E030E048ECEA
:1021700052E40E94CF26A70196010E94CF2621E0BB
:102180003EED42E45EE30E94D0276B017C0120E03B
:1021900030E048EC52E4C301B2010E94CF26AB010B
:1021A000BC0122E0CE0101960E94B70EBE016F5F16
:1021B0007F4F8CEE93E00E94720CCE0101960E943C
:1021C000BD0C43E050E06CEC71E08CEE93E00E94BB
:1021D000ED0C6CEE73E082EF93E00E94D00D6BEAA1
:1021E00071E0CE0101960E94F00D6CEE73E0CE011D
:1021F00001960E94380DBC018CEE93E00E94D00D38
:10220000CE0101960E94BD0C6FE172E084E094E083
:102210000E944B0D21E0B501A401CE0101960E9460
:10222000B70ECE0101960E94190DCE0101960E94B3
:10223000BD0C45E050E069E571E084E094E00E9467
:10224000ED0CA701960160E070E080E89FE30E943A
:10225000622620E03AE24DE257E40E941025AB01ED
:10226000BC0121E0CE0101960E94B70EBE016F5F56
:102270007F4FCE0107960E94E70D6FE571E0CE011A
:1022800007960E94220D0E94190DCE0107960E940A
:10229000BD0CCE0101960E94BD0C6CEE73E0CE0128
:1022A00001960E94E70D67E871E0CE0101960E9459
:1022B000220D64E074E00E94380DBC0184E094E0DB
:1022C0000E94D00DCE0101960E94BD0C65E070E029
:1022D00080E090E00E9404042C960FB6F894DEBFD4
:1022E0000FBECDBFDF91CF91FF90EF90DF90CF90E9
:1022F000BF90AF909F908F907F906F905F904F9026
:1023000008952F923F924F925F926F927F928F9299
:102310009F92AF92BF92CF92DF92EF92FF920F9374
:102320001F93CF93DF93CDB7DEB7C054D1090FB65B
:10233000F894DEBF0FBECDBF8C016CE471E084E089
:1023400094E00E949A0DC8010596059740F00C3E56
:102350002FEF120724F010936C0200936B020C3FD6
:102360004FEF140709F447C30CF059C0083F8FEF33
:102370001807C4F4063F9FEF1907ECF4053FAFEFD1
:102380001A070CF0B9C0013FBFEF1B07A4F4083EC9
:102390001F4F09F4CAC364E872E084E094E00E942D
:1023A0004B0D09C00B3FFFEF1F070CF015C3093F92
:1023B0001F4F0CF46EC18091080490910904892B81
:1023C00071F064E074E0CE0101960E94E70DCE0149
:1023D00001960E944D0ECE0101960E94BD0C64E64E
:1023E00070E080E090E00E940404C05CDF4F0FB614
:1023F000F894DEBF0FBECDBFDF91CF911F910F913B
:10240000FF90EF90DF90CF90BF90AF909F908F9014
:102410007F906F905F904F903F902F900895033082
:10242000110509F4EBC244F510161106ACF00F3F8C
:102430004FEF14070CF0BFCF0D3F1F4F09F0ABCF8C
:1024400081E08093740280916B0290916C02909372
:102450006F0280936E02AFCF0130110509F449C0BD
:102460000230110509F097CF80910101882309F40A
:10247000A2CF0E9483109FCF0A301105B4F406301A
:1024800011050CF098CF0430110509F433C3053061
:10249000110509F080CF69E772E084E094E00E94C2
:1024A0004B0D0E94BA04BC0135C30138110509F077
:1024B00072CF809101018823B1F00E94831064E003
:1024C00074E0CE0101960E94E70DCE0101960E94B4
:1024D0004D0ECE0101960E94BD0C64EF71E080E0CC
:1024E00090E00E94040464EF71E080E090E00E94BC
:1024F00004040E94ED0E5FCF60E080E10E94930330
:10250000809174028111C0C08AE090E0A0E0B0E048
:1025100021968CAF9DAFAEAFBFAF219762E272E064
:1025200084E094E00E944B0D312C212C1AAE1BAE9E
:10253000C12CD12C760102E310E0812C912C5401A6
:1025400080E10E94C403092E000CAA0BBB0B880E6D
:10255000991EAA1EBB1E65E070E080E090E00E941C
:1025600004040150110961F74090BC035090BD0371
:102570006090BE037090BF03C501B4010E94B124F6
:1025800020E030E040EA50E40E94102520E030E0F6
:1025900040E85AE30E94102520E030E048E452E48D
:1025A0000E94CF26A30192010E94622620E030E023
:1025B00040E751E40E9410254B015C01A301920108
:1025C0006AE979E989E390E40E9462269B01AC0103
:1025D000C501B4010E94CF2620E030E0A9010E948D
:1025E000632620E030E040E251E40E9410255B01C8
:1025F0008C01232D322D4AAD5BAD0E94CB271816DE
:1026000024F43A2C2B2C0AAF1BAF9FEFC91AD90A1E
:10261000E90AF90A21968CAD9DADAEADBFAD21970B
:102620008C159D05AE05BF050CF085CF6EE170E001
:1026300080E090E00E94040422E0432D522D6AAD18
:102640007BADCE0180960E94B70E61E671E0CE01AF
:1026500001960E94F00DBE01605E7F4FCE01019693
:102660000E94380D64E074E00E94380DBC0184E0E3
:1026700094E00E94D00DCE0101960E94BD0CCE01C7
:1026800080960E94BD0C97CE83E090E0A0E0B0E081
:102690003FCF0E9413054B015C0188E394E00E9448
:1026A000FF0564E670E080E090E00E940404109270
:1026B000530410925204109251041092500410923C
:1026C0004F0410924E048DE991E09093550480934D
:1026D000540490914404963108F047C02DEB30E04B
:1026E00030934F0420934E042BE931E03093510492
:1026F000209350042CE231E0309353042093520491
:102700002091680084E0983048F031E09E3008F471
:1027100030E081E001C0880F3A95EAF7822B809380
:1027200068002DE630E0983050F02BE630E09E3027
:1027300030F02CE630E0963110F030E020E03093BD
:102740004C0420934B04292F30E0983008F0B5C09A
:1027500081E001C0880F9A95EAF780934D0480913B
:102760005404909155040197F1F78091520490918F
:102770005304892B21F180915E0290915F02A4E0C5
:1027800088339A07E1F0009711F00E94FF058091CD
:1027900056048E7F8093560410925C0210925D0264
:1027A00088E394E090935F0280935E02E0914B0493
:1027B000F0914C04808190914D04892B808364E6D4
:1027C00070E080E090E00E9404041AAED12CC12C8D
:1027D000312C212C1CAE1BAE6CED462E65E0562E26
:1027E000612C712CFE01B096F9AFE8AF0E94130581
:1027F000681979098A099B09683B7B408105910525
:1028000008F072C088E394E00E949405892B09F4D3
:102810004DC040923C0450923D0460923E04709240
:102820003F040E94CD0597FD41C082349105C9F750
:102830008E010F5F1F4F78010E94CD0597FF4AC0A0
:1028400089818D3499F59801235E3F4F90E080E0B7
:10285000D8014D918D01840F911DA217B307C1F7C7
:102860008E5B9F4F2E8D30E0322F22274F8D240F0D
:10287000311D82179307D1F48C8190E0982F88271F
:102880002D81FC01E20FF11DFCAFEBAF2E80312C4E
:10289000322C22248F81280E311CC884D12CDC2CB0
:1028A000CC248985C80ED11CF1E0FAAF62E370E058
:1028B00080E090E00E94040499CF9E3040F42850BC
:1028C000310981E001C0880F2A95EAF746CF2E50E2
:1028D0003109F7CFD7018D937D01E8ADF9ADAE1782
:1028E000BF0709F0A9CFACCF0E9413056819790979
:1028F0008A099B09683B7B408105910598F44AADA4
:10290000442309F462C062E370E080E090E00E943A
:10291000040488E394E00E94FF0562E370E080E035
:1029200090E066C05AAD552309F44FC065E472E0EB
:1029300084E094E00E944B0DB601CE0180960E9487
:10294000A40DB101CE0186960E94A40D6BAD7CADA5
:10295000CE018C960E94A40D64E074E0CE01C29674
:102960000E94E70DBE01645D7F4FCE01C2960E94BA
:10297000380D67E871E00E94220DBE016A5D7F4F4D
:102980000E94380D67E871E00E94220DBE01605E72
:102990007F4F0E94380D65E671E00E94220DBC0158
:1029A00084E094E00E94D00DCE01C2960E94BD0C3E
:1029B000CE018C960E94BD0CCE0186960E94BD0C65
:1029C000CE0180960E94BD0C9ECF66E372E084E04B
:1029D00094E00E944B0D97CF80917402882321F0E0
:1029E00084E094E00E941F0268EC70E080E090E0D8
:1029F0000E940404E0CC10927402DDCC8BE0E82E3F
:102A0000F12C10E000E09924939493E2892E9092A7
:102A1000C7028092E9021092C8021092EA0262E0B4
:102A200083E20E94790710927A028093790288E803
:102A300093E00E945708D82EC12C88E893E00E94AA
:102A400057085C01AC28BD280E949206B50190E0B1
:102A500080E00E94AF242AE939E949E95FE30E9456
:102A6000CF260E9448270617170708F48B0162E358
:102A700070E080E090E00E94040481E0E81AF10830
:102A800031F665E572E084E094E00E944B0D19A2F6
:102A900018A21BA21AA21DA21CA24AE0BE016F5FCF
:102AA0007F4FC8010E94D820BE016F5F7F4FCE01CB
:102AB00080960E949A0D6BE671E0CE0101960E940D
:102AC000F00DBE01605E7F4FCE0101960E94380D71
:102AD00064E074E00E94380DBC0184E094E00E9440
:102AE000D00DCE0101960E94BD0CCE0180960E94B1
:102AF000BD0C13CF81E0809300010E94BA048C01C9
:102B000069E672E084E094E00E944B0D60E074E0BE
:102B1000601B710BCE0101960E94A40DCE0101969F
:102B20000E94190DCE010196ACCDF0E0E0E00995D0
:102B300042CC1F920F920FB60F9211242F933F9306
:102B40004F935F936F937F938F939F93AF93BF93B5
:102B5000EF93FF938BEE92E00E948902FF91EF9139
:102B6000BF91AF919F918F917F916F915F914F91A5
:102B70003F912F910F900FBE0F901F9018951F92AD
:102B80000F920FB60F9211242F938F939F93EF9371
:102B9000FF93E091FB02F091FC028081E091010340
:102BA000F091020382FD1BC09081809104038F5F2E
:102BB0008F7320910503821741F0E0910403F0E048
:102BC000E551FD4F958F80930403FF91EF919F9105
:102BD0008F912F910F900FBE0F901F9018958081AD
:102BE000F4CF1F920F920FB60F9211242F933F93A1
:102BF0008F939F93AF93BF938091610290916202F4
:102C0000A0916302B09164023091600223E0230F2F
:102C10002D3758F50196A11DB11D209360028093B8
:102C2000610290936202A0936302B0936402809168
:102C3000650290916602A0916702B09168020196C8
:102C4000A11DB11D8093650290936602A093670257
:102C5000B0936802BF91AF919F918F913F912F9157
:102C60000F900FBE0F901F90189526E8230F029625
:102C7000A11DB11DD2CF1F920F920FB60F9211243A
:102C80002F933F934F935F936F937F938F939F9374
:102C9000AF93BF93EF93FF93E0915E02F0915F02D9
:102CA000309749F0A685B7858585968D91FF14C02C
:102CB0009C918923A1F4FF91EF91BF91AF919F91D6
:102CC0008F917F916F915F914F913F912F910F90D5
:102CD0000FBE0F901F9018959C91892361F7A389CF
:102CE000B4899C918589809589238C93868997895D
:102CF0000197F1F7608D718DA685B785558538E010
:102D000020E0CB010197F1F7822F90E09595879510
:102D1000282F4C91452309F02068315091F7868D7A
:102D200081FD209580915C0290E001968F73992738
:102D300030915D02381799F0A0915C02B0E0A45E7A
:102D4000BD4F2C9380935C02828D938D0197F1F798
:102D5000A389B4898C919589892B8C93ACCF868D6E
:102D60008160868FF1CF1F920F920FB60F921124C0
:102D70002F933F934F935F936F937F938F939F9383
:102D8000AF93BF93EF93FF938091B900887F803614
:102D900009F44AC0F0F5883209F4A7C018F580316B
:102DA00009F49BC0B8F4882309F4F9C0883009F409
:102DB00094C0FF91EF91BF91AF919F918F917F91BF
:102DC0006F915F914F913F912F910F900FBE0F9098
:102DD0001F901895883109F488C0803251F780938C
:102DE000BF0214C0803409F49DC040F48033B9F3AD
:102DF0008833F9F68093BF0285ECB0C0803509F4C2
:102E000085C0883509F496C0883499F60E94140C60
:102E1000D0CF883909F48CC038F5883729F050F4C0
:102E2000883611F0803729F683E08093C102109232
:102E30001B0257C0883809F47BC0803919F08038EC
:102E400009F0B7CF80911B02803208F071C0E09189
:102E50001B0281E08E0F80931B028091BB00F0E08B
:102E6000E550FE4F80833DC0803B39F0E0F4803A6E
:102E700009F479C0883A09F09CCF84E08093C102BC
:102E80001092FA011092F901E0917702F091780224
:102E900009958091F90181110FC081E08093F901BA
:102EA0001092D90109C0803C09F4A6CF883C09F4EE
:102EB000A3CF883B09F07DCFE091FA0181E08E0F2E
:102EC0008093FA01F0E0E752FE4F80818093BB00CF
:102ED0009091FA018091F90129C080919C02809320
:102EE000BB0085EC8093BC0064CF9091BE028091C2
:102EF000BD02981758F5E091BE0281E08E0F8093D5
:102F0000BE02F0E0E356FD4F8081E9CFE091BE02C2
:102F100081E08E0F8093BE028091BB00F0E0E3560B
:102F2000FD4F80839091BE028091BD029817C8F238
:102F300085E8D8CFE091BE0281E08E0F8093BE027B
:102F40008091BB00F0E0E356FD4F80838091C0028A
:102F500081115CCF81E080939B0284EA8093BC0066
:102F60001092C10226CF85EC8093BC001092C10262
:102F700080911B02803230F4E0911B02F0E0E550BA
:102F8000FE4F108260911B0270E0E0917502F0919B
:102F900076028BEF91E0099510921B020ACF1092F6
:102FA000BF0234CF1092EE021092ED0288EE93E051
:102FB000A0E0B0E08093EF029093F002A093F102C2
:102FC000B093F20228E131E03093EC022093EB025F
:102FD00025EC30E03093F8022093F70224EC30E047
:102FE0003093FA022093F90220EC30E03093FC0297
:102FF0002093FB0221EC30E03093FE022093FD028F
:1030000022EC30E0309300032093FF0226EC30E006
:1030100030930203209301031092040310920503DE
:10302000109206031092070310928B0310928A03EA
:1030300080938C0390938D03A0938E03B0938F03A2
:103040002AE231E0309389032093880310926404CC
:1030500010923B0410923A0480933C0490933D04F8
:10306000A0933E04B0933F048CE391E09093390425
:103070008093380410924F0410924E041092510421
:10308000109250041092530410925204109255045E
:1030900010925404609156046E7F6D7F60935604C5
:1030A0006695617081E0682789E00E94650361E0B0
:1030B00089E00E949303EBE7F3E0E491E093480496
:1030C000E7E6F3E0E491F0E0EE0FFF1FEC5AFC4F6F
:1030D0008591949190934A048093490460E08AE03A
:1030E0000E9493038091560481FD04C061E08AE050
:1030F0000E9465038AE080934404ECE7F3E0E491E6
:10310000E0934504E8E6F3E0E491F0E0EE0FFF1F02
:10311000E65BFC4F8591949190934704809346041D
:103120008FEF80931304809314048093150480938D
:1031300016046CE471E084E094E00E94F00D6CE40D
:1031400071E08EEF93E00E94F00D6CE471E088EF87
:1031500093E00E94F00D6CE471E082EF93E00E9436
:10316000F00D6CE471E08CEE93E00E94F00D6EE6E1
:1031700071E086EE93E00E94F00D65E771E080EE6D
:1031800093E00E94F00D86E190E090939503809388
:1031900094038CE79CE8A1E0B0E08093A0039093B7
:1031A000A103A093A203B093A30381EA97E6A3E34C
:1031B000BDEB8093A4039093A503A093A603B093C3
:1031C000A70386E696E6A6EABFE38093A80390935A
:1031D000A903A093AA03B093AB0381E08093B40347
:1031E00029E130E03093B6032093B5038093B70311
:1031F00080E090E4ACE1B5E48093B8039093B90328
:10320000A093BA03B093BB031092BC031092BD030A
:103210001092BE031092BF03E0ECF3E080E1DF0107
:103220001D928A95E9F71092D0031092D103109263
:10323000D2031092D3031092D4031092D5031092AC
:10324000D6031092D7031092D8031092D90310928C
:10325000DA031092DB031092DC031092DD0310926C
:10326000DE031092DF030895CF93DF93CDB7DEB76F
:103270002C970FB6F894DEBF0FBECDBF789484B5FF
:10328000826084BD84B5816084BD85B5826085BD62
:1032900085B5816085BD80916E00816080936E00F0
:1032A00010928100809181008260809381008091E2
:1032B0008100816080938100809180008160809393
:1032C00080008091B10084608093B1008091B00053
:1032D00081608093B00080917A00846080937A004E
:1032E00080917A00826080937A0080917A00816078
:1032F00080937A0080917A00806880937A0010929F
:10330000C10061E08EE00E949303E091FB02F09126
:10331000FC0282E08083E091F702F091F8021082D3
:10332000E091F902F091FA028FEC8083109203038E
:10333000E091FF02F091000386E08083E091FD02BE
:10334000F091FE02808180618083E091FD02F09126
:10335000FE02808188608083E091FD02F091FE0290
:10336000808180688083E091FD02F091FE0280817F
:103370008F7D808360E08EE00E9465030E945A0684
:1033800081E08093C70283E28093E9021092C80231
:103390001092EA0260E188E893E00E949E080E9491
:1033A00092068FE39CE90197F1F700C0000068ECFA
:1033B00070E080E090E00E94040484E690E0909346
:1033C0000301809302010E94D1258093690285E662
:1033D00090E00E94D12580936A02009169021091C9
:1033E0006A02B801012E000C880B990B0E94B124CF
:1033F0009B01AC010E942028811106C00B501109CD
:103400000C30110508F4B4C084E690E00E94E70B8C
:1034100068EC70E080E090E00E94040468EA72E0EA
:1034200084E094E00E944B0D64E074E0CE010196CC
:103430000E94E70DCE0101960E944D0ECE0101962D
:103440000E94BD0C0E945A0664E670E080E090E0A5
:103450000E94040486E780930A04809113048F3F3E
:1034600011F40E945A06809113048F3F01F5809158
:103470000A0491E09093C7028093E9021092C80277
:103480001092EA0260ED88E893E00E949E080E9494
:10349000920661E080910A040E94790710927A02F4
:1034A0008093790288E893E00E945708F82EF8E5A7
:1034B000FF1609F488C06CE972E084E094E00E9491
:1034C0004B0D1092010164E074E0CE0101960E9460
:1034D000E70DCE0101960E944D0ECE0101960E948D
:1034E000BD0C98EE892E93E0992EA12CB12C712C55
:1034F000612C2AE2E22EF12C80E0C82E80E0D82E4A
:103500006CE471E0CE0107960E94F00D10E08BEEA6
:1035100092E00E946902181619060CF0C5C011113C
:10352000C3C08BEE92E00E9447028A3009F00EC1C0
:1035300010916D02112309F41EC18091FC0390913A
:10354000FD03892B09F410C160E871E0CE010196FA
:103550000E94F00DBE01695F7F4FCE0101960E946F
:10356000380D0E941F02CE0101960E94BD0CFCC0C6
:1035700034E9C32E33E0D32E04E610E0C8010E94E4
:10358000D125F60181936F010F5F1F4F003B11059D
:10359000A9F78091940390919503909305018093EE
:1035A000040166E973E0CE0101960E94F00DBE01B0
:1035B0006F5F7F4F86EE93E00E94720CCE01019602
:1035C0000E94BD0C25CF88E80E94B60B909318048A
:1035D000809317048AE80E94B60B90931A04809394
:1035E00019048CE80E94B60B90931C0480931B0472
:1035F0008EE80E94B60B90931E0480931D0480E910
:103600000E94B60B9093200480931F0482E90E94CD
:10361000B60B909322048093210484E90E94B60B98
:10362000909324048093230486E90E94B60B909320
:1036300026048093250488E90E94B60B9093280401
:10364000809327048AE90E94B60B90932A04809302
:1036500029048CE90E94B60B90932C0480932B04D0
:103660008EE90E94B60B90932E0480932D048091D6
:1036700013048F3F09F035CF80910A0491E09093B5
:10368000C7028093E9021092C8021092EA0264EF26
:1036900088E893E00E949E086FE388E893E00E9428
:1036A0009E080E9492061DCF8B859C85892B51F028
:1036B0008BEE92E00E94F80264E170E080E090E01E
:1036C0000E940404BE01695F7F4F88EF93E00E946F
:1036D000720CCE0107960E94BD0C6CE471E084E090
:1036E00094E00E949A0D8091FC039091FD0381303B
:1036F000910509F0C8C068EF73E0CE0101960E9401
:10370000E70D8D819E81892B99F0E981FA813097AF
:1037100079F08081823409F44DC07CF58A3209F455
:10372000AFC0813409F43FC062E971E08332E9F14E
:10373000BE016F5F7F4F88EF93E00E94D00D6AE07B
:1037400070E080E090E00E94040440C08D3009F4F5
:10375000EFCE89831A8241E050E0BE016F5F7F4F58
:10376000CE0107960E94ED0C6AE070E080E090E0E8
:103770000E940404CCCE11E0F7CF8136A1F074F49E
:103780008334B1F66FE871E088EF93E00E949A0D00
:1037900021E0209374028DEF9FEF16C0823651F026
:1037A000833681F3C5CF69E871E088EF93E00E942A
:1037B0009A0D0CC06CE871E088EF93E00E949A0DBE
:1037C000109274028CEF9FEF0E948111CE0101963E
:1037D0000E94BD0C88EF93E00E944C0CCB010E942C
:1037E000811180917402882309F43EC00E94130560
:1037F000A50194010E943126CA01B9010E94AF249B
:1038000020917002309171024091720250917302C6
:103810000E94622620910A0130910B0140910C0117
:1038200050910D010E94CB271816F4F40E94130545
:10383000A50194010E943126CA01B9010E94AF245A
:10384000609370027093710280937202909373027E
:1038500080916E0290916F020E9481116AE070E087
:1038600080E090E00E940404C114D10409F448CE21
:103870000E947502882309F443CE0E9400003CCECA
:1038800065E971E092CF049768F568E971E0CE01CF
:1038900001960E94F00DBE016F5F7F4F88EF93E0AD
:1038A0000E94570C182FCE0101960E94BD0C1123C7
:1038B000C9F08091FC039091FD03029788F0E0919C
:1038C000F803F091F903309759F0818180330CF4BB
:1038D000845EF701E81BF10987FDF395CF017FCFE7
:1038E00080E0F6CF68EF73E08EEF93E00E94D00D9A
:1038F0000091FE031091FF030115110571F0F8010D
:1039000081918F01882349F0082E000C990B0E94A9
:10391000C62CF80131978083F2CF6FE273E0CE01BD
:1039200001960E94700DBE016F5F7F4F8EEF93E096
:103930000E94570C182FCE0101960E94BD0C112336
:1039400019F0F30109954DCF67E273E0CE010196BE
:103950000E94700DBE016F5F7F4F8EEF93E00E945B
:10396000570C182FCE0101960E94BD0C112399F11E
:103970006AE971E0CE0101960E94F00D60EE73E0FD
:10398000CE0101960E94380DBC0184E094E00E94B3
:10399000D00DCE0101960E94BD0C64EA71E0CE010B
:1039A00001960E94F00D64E074E0CE0101960E9441
:1039B000380DBC01CE0107960E94E70DCE01079697
:1039C0000E944D0ECE0107960E94BD0CCE010196BD
:1039D0000E94BD0C06CF60E273E0CE0101960E940A
:1039E000700DBE016F5F7F4F8EEF93E00E94570C0A
:1039F000182FCE0101960E94BD0C112359F062E1EF
:103A000073E084E094E00E944B0D86EE93E00E9408
:103A1000190DC3CF6BE073E0CE0101960E94700DCB
:103A2000BE016F5F7F4F8EEF93E00E94570C182FFF
:103A3000CE0101960E94BD0C112311F127E030E068
:103A400046E050E068EF73E0CE0101960E94010E5F
:103A5000BE016F5F7F4F82EF93E00E94720CCE0138
:103A600001960E94BD0C82EF93E00E944C0C672BE4
:103A700019F410926D02B5CEF1E0F0936D02B1CE63
:103A800064E073E0CE0101960E94700DBE016F5F8D
:103A90007F4F8EEF93E00E94570C182FCE010196B6
:103AA0000E94BD0C112309F47BC02091FC033091CE
:103AB000FD032730310508F494CE46E050E068EF6E
:103AC00073E0CE0101960E94010EBE016F5F7F4F31
:103AD00082EF93E00E94720CCE0101960E94BD0C11
:103AE0008091F2039091F303009709F455C00E946E
:103AF0007D2060930A0170930B0180930C019093D9
:103B00000D0169EF72E084E094E00E944B0D40915A
:103B10000A0150910B0160910C0170910D0122E09E
:103B2000CE0101960E94B70EBE016F5F7F4FCE019E
:103B300007960E94E70D66EA71E0CE0107960E94A3
:103B4000220D0E94190DCE0107960E94BD0CCE01D8
:103B500001960E94BD0C64E074E0CE0101960E94C3
:103B6000E70DCE0101960E944D0ECE0101960E94F6
:103B7000BD0C0E941305A50194010E943126CA01C3
:103B8000B9010E94AF246093700270937102809318
:103B900072029093730225CE60E070E0CB01A9CF52
:103BA00062EF72E0CE0101960E94700DBE016F5F60
:103BB0007F4F8EEF93E00E94570C182FCE01019695
:103BC0000E94BD0C112309F469C02091FC033091BF
:103BD000FD032730310508F404CE46E050E068EFDD
:103BE00073E0CE0101960E94010EBE016F5F7F4F10
:103BF00082EF93E00E94720CCE0101960E94BD0CF0
:103C00008091F2039091F303009709F443C00E945E
:103C10007D206093060170930701809308019093C3
:103C2000090167EE72E084E094E00E944B0D409140
:103C3000060150910701609108017091090121E08E
:103C4000CE0101960E94B70EBE016F5F7F4FCE017D
:103C500007960E94E70D66EA71E0CE0107960E9482
:103C6000220D0E94190DCE0107960E94BD0CCE01B7
:103C700001960E94BD0C64E074E0CE0101960E94A2
:103C8000E70DCE0101960E944D0ECE0101960E94D5
:103C9000BD0CA7CD60E070E0CB01BBCF62EE72E05F
:103CA000CE0101960E94700DBE016F5F7F4F8EEFB7
:103CB00093E00E94570C182FCE0101960E94BD0C74
:103CC000112341F126E030E044E050E068EF73E07A
:103CD000CE0101960E94010EBE016F5F7F4F82EF01
:103CE00093E00E94720CCE0101960E94BD0C82EFFF
:103CF00093E00E944C0C709395036093940370932F
:103D000005016093040180910201909103010E94DA
:103D1000E70B67CD6EED72E0CE0101960E94700D4B
:103D2000BE016F5F7F4F8EEF93E00E94570C182FFC
:103D3000CE0101960E94BD0C112309F451C02091BF
:103D4000FC033091FD0343E050E068EF73E0CE01E7
:103D500001960E94010EBE016F5F7F4F82EF93E0DC
:103D60000E94720CCE0101960E94BD0C62EF73E0BE
:103D7000CE0101960E94E70D1F82188641E050E0B7
:103D8000BE01695F7F4FCE0101960E94ED0C81114B
:103D900004C0CE0101960E94AB0CBE016F5F7F4F45
:103DA00086EE93E00E94D00DCE0101960E94BD0CDC
:103DB0000091EA031091EB030115110509F4A3CF5B
:103DC000015011096091E6037091E703A80186E9AB
:103DD00093E00E94EC2CF801EA56FC4F108293CF3E
:103DE0006BED72E0CE0101960E94700DBE016F5F17
:103DF0007F4F8EEF93E00E94570C182FCE01019653
:103E00000E94BD0C112309F48CC02091FC03309159
:103E1000FD032031310508F0E4CC42E050E068EFCA
:103E200073E0CE0101960E94010EBE016F5F7F4FCD
:103E300082EF93E00E94720CCE0101960E94BD0CAD
:103E40008091F2039091F303009799F10E947D20F5
:103E500020E030E048EC52E40E9410250E94412707
:103E60006093A0037093A1038093A2039093A30394
:103E70008B019C0100591F452140310901341C4927
:103E800021053105D0F068EA71E0CE0101960E946B
:103E9000F00D62EF73E0CE0101960E94380D6EEADC
:103EA00071E00E94220DBC0184E094E00E94D00DDC
:103EB0008DCD60E070E0CB01CBCF0E94B12420E03B
:103EC00030E048EC52E40E94CF26AB01BC0122E076
:103ED000CE0101960E94B70EBE016F5F7F4F84E056
:103EE00094E00E94720CCE0101960E94BD0C6EEB14
:103EF00071E0CE0101960E94F00D64E074E0CE0105
:103F000001960E94380D6BEC71E00E94220DBC01FD
:103F100084E094E00E94D00DCE0101960E94BD0C79
:103F2000F2CE60ED71E0CE0101960E94F00DBE016F
:103F30006F5F7F4F8EEF93E00E94570C182FCE01DA
:103F400001960E94BD0C112309F45EC009E110E046
:103F5000212C312C210180E10E94C403BC01990F66
:103F6000880B990B0E94B1249B01AC01C201B101E5
:103F70000E9463261B012C016AE070E080E090E063
:103F80000E9404040150110931F720E030E040EABA
:103F900050E4C201B1010E94102520E030EC4FE74F
:103FA00054E40E94CF2620E030E048EC51E40E9427
:103FB000CF266093BC037093BD038093BE039093A0
:103FC000BF0380910201909103010E94E70B68EC0E
:103FD00072E084E094E00E944B0D4091BC0350914C
:103FE000BD036091BE037091BF0322E0CE01019634
:103FF0000E94B70EBE016F5F7F4FCE0107960E94F1
:10400000E70D64ED71E029CE64EC72E0CE0101961B
:104010000E94700DBE016F5F7F4F8EEF93E00E9494
:10402000570C182FCE0101960E94BD0C112309F4E4
:10403000D8CB2091FC033091FD0343E050E068EFC2
:1040400073E0CE0101960E94010EBE016F5F7F4FAB
:1040500082EF93E00E94720CCE0101960E94BD0C8B
:1040600082EF93E00E944C0C70936C0260936B02A1
:10407000B8CB80EE93E00E94BD0C86EE93E00E94E8
:10408000BD0C8CEE93E00E94BD0C82EF93E00E9489
:10409000BD0C88EF93E00E94BD0C8EEF93E00E9470
:1040A000BD0C84E094E00E94BD0C8CE391E0909301
:1040B00039048093380488E394E00C94FF05EF9270
:1040C0000F931F93CF93DF93E80134E047FD34E172
:1040D000042E000C550B57FF03C051954195510913
:1040E000E32E022F242FAE010E94F220CE01DF9199
:1040F000CF911F910F91EF900895662777270C9429
:1041000051221F93FC0199278827BC01E894119143
:104110001032E9F3193010F01E30C8F31B3251F0A1
:104120001D3249F4689406C00E94C320610F711DBE
:10413000811D911D119110531A30B0F33EF49095EA
:104140008095709561957F4F8F4F9F4F1F91089578
:10415000FB01DC0105900D920020E1F70895FC01C0
:1041600005900020E9F7809590958E0F9F1F089588
:10417000BB274A3031F4992322F4BDE29095819512
:104180009F4F0C94D920592F482F372F262F660F79
:10419000771F881F991F660F771F881F991F620F4F
:1041A000731F841F951F660F771F881F991F08951F
:1041B000BB27FB015527AA27880F991FAA1FA41701
:1041C00010F0A41B83955051B9F7A05DAA3308F0F5
:1041D000A95DA193009779F7B111B1931192CB0129
:1041E0000C949A24A9E0B0E0E8EFF0E20C940026E9
:1041F0006A01F22EB02E102FFBE3AF2EA01608F4AA
:104200001BE31F5F012F27E0AE014F5F5F4F0E944E
:10421000A123BC018981982F9970913009F43FC086
:104220009BE2E1FC04C09E2D9170E0FC3AC05E2D43
:104230005071E82FE87083FF46C084E0911101C0FF
:1042400083E0EF2DE81B8F1508F0E0E0D6018E2FFC
:1042500020E2552351F1992329F0D6019C93C60100
:1042600001966C0196012D5F3F4FE2FE24C08EE463
:10427000D6018C9391E411969C93119712968C938E
:10428000D9018E2F90E281111BC0E20FF32FF11D97
:1042900010828EEF9FEF2996ECE00C941C269DE295
:1042A000C6CF90E2C4CF2D9381508111FCCFCE0EAA
:1042B000D11CE0E0D0CF8EE6D6018C9391E6DBCF27
:1042C0009D938150E0CF482F447082FF3DC084E031
:1042D000911101C083E08F1510F4EF2DE81BD6017A
:1042E0008E2F20E2552309F1992329F0D6019C93C2
:1042F000C60101966C0196012D5F3F4FE2FE1BC087
:1043000089E4D6018C938EE411968C93119786E400
:1043100012968C93D9018E2F90E2882309F4B5CFA1
:104320009D938150FACF2D9381508111FCCFCE0EF9
:10433000D11CE0E0D9CF89E6D6018C938EE61196A8
:104340008C93119786E6E4CF9B0177FF02C030E0A3
:1043500020E0A1E0B0E0911102C0B0E0A0E0F901DE
:104360003196AE0FBF1F8B2C912CBB2009F461C07E
:104370005401EFEFAE1ABE0AAA0DBB1DFA161B06BA
:1043800019F014F04F2D4A1B511188C0E3FC59C09D
:104390007601A42FB0E2A1114FC0C40ED11C992305
:1043A00009F45BC040E0D6011196F60190836D01DF
:1043B000552309F448C0012F060F9A81582F5071D8
:1043C00084FF03C0913309F4015010160CF047C06C
:1043D000093008F008E0EEE2FE2E5B01A01AB108F9
:1043E00085019194819491082F3F320729F4D601D9
:1043F000FC92F60131966F016217730794F1021770
:1044000013077CF5DB01A21BB30BAA24A394B12CE8
:10441000AC0EBD1EAA0DBB1D11968C912150310909
:10442000D601119628153905F4F0F60180836D0147
:10443000DBCFB12CA12CA0CFF701B1937F01A1500C
:10444000AACF9111B0CFD601942F50E302C05D9353
:1044500091509111FCCFC40ED11C40E0ACCF01E0D3
:10446000BACF80E3DBCF6217730731F4963388F459
:10447000953311F4552369F0F6018083FD01842FF3
:1044800090E2811108C0A40FB11D1C9290E080E061
:1044900002CF81E3F1CF91938150F3CF911183CF7C
:1044A0008ACFB0E0A0E0E7E5F2E20C9400265C01E0
:1044B0007B016115710519F0DB018D939C938501DA
:1044C0000F5F1F4FF501D0818D2F90E00E9479245E
:1044D0006C01892BB9F5DD32B9F50F5F1F4FD5019E
:1044E0001196DC91C1E05801F1E0AF1AB10843E048
:1044F00050E062EF70E0C5010E948224892B69F5CB
:10450000680182E0C80ED11C45E050E06DEE70E01D
:10451000C6010E948224892B21F4680197E0C90E0C
:10452000D11CE114F10419F0D701CD92DC9260E0C6
:1045300070E080E89FEFC111FFC060E070E080E8AC
:104540009FE7FAC05801BBCFDB3229F485010E5F2B
:104550001F4FF501D181C0E0C6CF43E050E06AEEC5
:1045600070E0C5010E948224892BE9F0F80110E077
:1045700000E020E030E0A9015F01B0ED8B2E8D0E50
:1045800089E08815C8F19C2E689491F88C2F88706A
:10459000C2FF16C0811102C00F5F1F4F3196D501B7
:1045A000DC91C92DE9CFE114F10429F00E5F1F4F12
:1045B000F7011183008360E070E080EC9FE7BCC0EE
:1045C000882311F001501109A5E0B0E00E94E72511
:1045D0009B01AC01220F331F441F551F280D311DB5
:1045E000411D511D283999E93907490799E15907B2
:1045F000A8F2C6609C2ED2CFAEEF8A1206C0C3FDD1
:104600003CC09C2E689493F8C9CFDF7DD534A9F5C2
:1046100080818D3239F4C061DF011296818162E0C0
:1046200070E006C0DF018B32C1F3119661E070E0EB
:1046300080535D01A61AB70A8A30F8F4E0E8CE1676
:10464000ECE0DE065CF4B601660F771F660F771F9D
:10465000C60ED71ECC0CDD1CC80ED11C5D01FFEFB1
:10466000AF1ABF0A8C9180538A30A8F1C4FF03C0EF
:10467000D194C194D1080C0D1D1DC1FF09C0E114D6
:10468000F10431F081E0A81AB108D701AD92BC92D3
:10469000CA01B9010E94AF24C370C33009F4905815
:1046A0004B015C0120E030E0A9010E94AA2488238C
:1046B00009F440C0C1E2D1E017FF05C01195019592
:1046C0001109C9E0D1E06E01B8E1CB1AD10880E24E
:1046D000E82EF12C0FC0D501B1CFFE012591359107
:1046E000459154910E191F09C501B4010E9410256E
:1046F0004B015C01D501C4010E151F0574F7249709
:10470000F594E794CC16DD06A9F78A2F880F8B2F36
:10471000881F8F3F49F020E030E0A901C501B401B6
:104720000E94AA24811106C082E290E09093660460
:1047300080936504C501B401CDB7DEB7ECE00C94FD
:104740001C26283008F027E03327DA01990F311DA5
:1047500087FD916000966105710539F432602E5F26
:104760003D9330E32A95E1F708959F3F30F080387C
:104770007105610509F03C5F3C5F3D93913008F0A5
:104780008068911DDF93CF931F930F93FF92EF9259
:10479000192F987F9695E92F96959695E90FFF2703
:1047A000E158FE4F99273327EE24FF24A701E701A4
:1047B00005900894079428F4360FE71EF81E491F49
:1047C000511D660F771F881F991F0694A1F705904A
:1047D000079428F4E70EF81E491F561FC11D770FD6
:1047E000881F991F661F0694A1F70590079428F467
:1047F000F80E491F561FC71FD11D880F991F661F2E
:10480000771F0694A1F70590079420F4490F561FCF
:10481000C71FD81F990F661F771F881F0694A9F717
:1048200084911095177041F0D695C7955795479587
:10483000F794E7941A95C1F7E5E2F1E068941590D2
:10484000159135916591959105907FE27395E118E9
:10485000F10A430B560BC90BD009C0F7E10CF11E4E
:10486000431F561FC91FD01D7EF4703311F48A9563
:10487000E6CFE894015030F0080F0AF40027021741
:1048800008F4202F2395022F7A3328F079E37D93C3
:104890002A95E9F710C07D932A9589F60694979595
:1048A0006795379517951794E118F10A430B560B46
:1048B000C90BD00998F023957E9173957A3308F04F
:1048C00070E37C932013B8F77E9170617D9330F094
:1048D000839571E37D9370E32A95E1F71124EF90BE
:1048E000FF900F911F91CF91DF91992787FD9095B0
:1048F000089591110C947D25803219F089508550CE
:10490000C8F70895FB01DC014150504088F08D91BB
:1049100081341CF08B350CF4805E659161341CF0A1
:104920006B350CF4605E861B611171F3990B089571
:10493000881BFCCFDC01FC01672F71917723E1F725
:10494000329704C07C916D9370836291AE17BF075C
:10495000C8F308950E94EC2408F481E00895E894D7
:1049600009C097FB3EF490958095709561957F4FB7
:104970008F4F9F4F9923A9F0F92F96E9BB27939565
:10498000F695879577956795B795F111F8CFFAF475
:10499000BB0F11F460FF1BC06F5F7F4F8F4F9F4FA6
:1049A00016C0882311F096E911C0772321F09EE804
:1049B000872F762F05C0662371F096E8862F70E06A
:1049C00060E02AF09A95660F771F881FDAF7880F44
:1049D0009695879597F90895990F0008550FAA0B9A
:1049E000E0E8FEEF16161706E807F907C0F0121602
:1049F0001306E407F50798F0621B730B840B950B05
:104A000039F40A2661F0232B242B252B21F4089559
:104A10000A2609F4A140A6958FEF811D811D0895F6
:104A20000E9423250C9497250E94892538F00E9426
:104A3000902520F0952311F00C9480250C94862568
:104A400011240C94CB250E94A82570F3959FC1F3E7
:104A5000950F50E0551F629FF001729FBB27F00D2C
:104A6000B11D639FAA27F00DB11DAA1F649F662781
:104A7000B00DA11D661F829F2227B00DA11D621FD0
:104A8000739FB00DA11D621F839FA00D611D221F8A
:104A9000749F3327A00D611D231F849F600D211D6E
:104AA000822F762F6A2F11249F5750409AF0F1F0F1
:104AB00088234AF0EE0FFF1FBB1F661F771F881F5A
:104AC00091505040A9F79E3F510580F00C948025ED
:104AD0000C94CB255F3FE4F3983ED4F3869577950D
:104AE0006795B795F795E7959F5FC1F7FE2B880F00
:104AF000911D9695879597F9089599278827089588
:104B000097F99F6780E870E060E008959FEF80EC80
:104B1000089500240A941616170618060906089523
:104B200000240A9412161306140605060895092E89
:104B30000394000C11F4882352F0BB0F40F4BF2BF8
:104B400011F460FF04C06F5F7F4F8F4F9F4F089538
:104B500057FD9058440F551F59F05F3F71F047952E
:104B6000880F97FB991F61F09F3F79F08795089513
:104B7000121613061406551FF2CF4695F1DF08C032
:104B8000161617061806991FF1CF8695710561054F
:104B900008940895E894BB2766277727CB0197F9F7
:104BA0000895F999FECF92BD81BDF89A992780B5F5
:104BB0000895262FF999FECF1FBA92BD81BD20BD61
:104BC0000FB6F894FA9AF99A0FBE019608950E94CA
:104BD0005326A59F900DB49F900DA49F800D911D0D
:104BE00011240895B7FF0C94E7250E94E725821B46
:104BF000930B08952F923F924F925F926F927F9204
:104C00008F929F92AF92BF92CF92DF92EF92FF92DC
:104C10000F931F93CF93DF93CDB7DEB7CA1BDB0B88
:104C20000FB6F894DEBF0FBECDBF09942A8839882D
:104C300048885F846E847D848C849B84AA84B98434
:104C4000C884DF80EE80FD800C811B81AA81B98140
:104C5000CE0FD11D0FB6F894DEBF0FBECDBFED0154
:104C60000895A1E21A2EAA1BBB1BFD010DC0AA1FAD
:104C7000BB1FEE1FFF1FA217B307E407F50720F0C5
:104C8000A21BB30BE40BF50B661F771F881F991F40
:104C90001A9469F760957095809590959B01AC0189
:104CA000BD01CF010895A29FB001B39FC001A39F92
:104CB000700D811D1124911DB29F700D811D112455
:104CC000911D08955058BB27AA270E947A260C945C
:104CD00097250E94892538F00E94902520F039F40C
:104CE0009F3F19F426F40C9486250EF4E095E7FB1B
:104CF0000C948025E92F0E94A82558F3BA17620763
:104D000073078407950720F079F4A6F50C94CA255B
:104D10000EF4E0950B2EBA2FA02D0B01B9019001D6
:104D20000C01CA01A0011124FF27591B99F0593F1A
:104D300050F4503E68F11A16F040A22F232F342F62
:104D40004427585FF3CF469537952795A795F040B0
:104D50005395C9F77EF41F16BA0B620B730B840BC5
:104D6000BAF09150A1F0FF0FBB1F661F771F881F7D
:104D7000C2F70EC0BA0F621F731F841F48F48795D5
:104D800077956795B795F7959E3F08F0B0CF9395C7
:104D9000880F08F09927EE0F9795879508950E9440
:104DA000E3260C9497250E94902558F00E948925AF
:104DB00040F029F45F3F29F00C94802551110C94A8
:104DC000CB250C9486250E94A82568F39923B1F37E
:104DD000552391F3951B550BBB27AA276217730721
:104DE000840738F09F5F5F4F220F331F441FAA1FB5
:104DF000A9F335D00E2E3AF0E0E832D09150504071
:104E0000E695001CCAF72BD0FE2F29D0660F771F1E
:104E1000881FBB1F261737074807AB07B0E809F004
:104E2000BB0B802DBF01FF2793585F4F3AF09E3F89
:104E3000510578F00C9480250C94CB255F3FE4F36A
:104E4000983ED4F3869577956795B795F7959F5FCC
:104E5000C9F7880F911D9695879597F90895E1E018
:104E6000660F771F881FBB1F621773078407BA0777
:104E700020F0621B730B840BBA0BEE1F88F7E095D2
:104E800008950E9448276894B1110C94CB25089589
:104E90000E94B02588F09F5798F0B92F9927B751F5
:104EA000B0F0E1F0660F771F881F991F1AF0BA95CE
:104EB000C9F714C0B13091F00E94CA25B1E008953D
:104EC0000C94CA25672F782F8827B85F39F0B93F2F
:104ED000CCF3869577956795B395D9F73EF4909581
:104EE0008095709561957F4F8F4F9F4F089597FBE9
:104EF00016F40E94BB270C947E27E894F92F96EBBA
:104F0000FF2381F0121613061406440B9395F695B1
:104F100087957795679557954040FF23B9F71BC054
:104F200099270895882351F49850D2F7872B762F2C
:104F3000652F542F432F322F20E0B1F312161306A2
:104F40001406440B88233AF09A95440F551F661FA8
:104F5000771F881FCAF755234AF4440F551F11F4D1
:104F600060FF04C06F5F7F4F8F4F9F4F880F9695F4
:104F7000879597F9089590958095709560955095CF
:104F80004095309521953F4F4F4F5F4F6F4F7F4F6B
:104F90008F4F9F4F08950E94EC2408F48FEF0895DF
:104FA000FA01EE0FFF1F309621053105A1F16115C1
:104FB000710561F48038BFE39B0749F1689490382C
:104FC000810561F08038BFEF9B0741F099234AF5D6
:104FD000FF3FE1053105210519F1E8940894E795B3
:104FE000D901AA2329F4AB2FBE2FF85FD0F310C04C
:104FF000FF5F70F4A695E0F7F73950F019F0FF3A2B
:1050000038F49F779F930DD00F9007FC9058089528
:1050100046F00C94862560E070E080E89FE30895F8
:105020004FE79F775F934F933F932F930E94D02832
:105030002F913F914F915F910E9410250C942D2844
:105040000E94EC24880B990B089529F416F00C9417
:1050500080250C94CA250C9486250E94B025A8F3BF
:105060009638A0F707F80F92E8942BE33AEA48EB5A
:105070005FE70E9426250F920F920F924DB75EB701
:105080000F920E941829E8E6F0E00E945F284F91F5
:105090005F91EF91FF91E595EE1FFF1F49F0FE57DD
:1050A000E0684427EE0F441FFA95E1F74195550B50
:1050B0000E9492280F9007FE0C9486280895DF9393
:1050C000CF931F930F93FF92EF92DF927B018C019E
:1050D000689406C0DA2EEF010E942325FE01E894B1
:1050E000A5912591359145915591A6F3EF010E9427
:1050F0007A26FE019701A801DA9469F7DF90EF9014
:10510000FF900F911F91CF91DF9108959B01AC010A
:1051100060E070E080E89FE30C94CF260C9480253B
:105120000C944C290E94B025D8F39923C9F3940F0D
:10513000511DA3F39150504094F059F0882332F060
:10514000660F771F881F91505040C1F79E3F510551
:105150002CF7880F911D9695879597F908955F3FD5
:10516000ACF0983E9CF0BB27869577956795B795F0
:1051700008F4B1609395C1F7BB0F58F711F460FFC5
:10518000E8CF6F5F7F4F8F4F9F4FE3CF0C94CB25BE
:1051900016F00C944C290C94862568940C94802568
:1051A0000E94B025A8F39923C1F3AEF3DF93CF9308
:1051B0001F930F93FF92C92FDD2788232AF0219791
:1051C000660F771F881FDAF720E030E040E85FEBDA
:1051D0009FE3883920F0803E38F021968F770E9437
:1051E0006326E0E9F0E004C00E946326EDEBF0E006
:1051F0000E945F288B01BE01EC01FB2E6F577109E5
:105200007595771F880B990B0E94B12428E132E72E
:1052100041E35FE30E942325AF2D9801AE01FF908B
:105220000F911F91CF91DF910E947A260C949725C0
:10523000FA01DC01AA0FBB1F9B01AC01BF5728F488
:10524000222733274427507820C0B75190F4AB2F42
:105250000024469537952795011CA395D2F300208D
:1052600071F0220F331F441FB395DAF30ED00C9464
:10527000622661307105A0E88A07B94630F49B01C7
:10528000AC016627772788279078309621F0208315
:1052900031834283538308959F3F31F0915020F42E
:1052A000879577956795B795880F911D9695879502
:1052B00097F90895DB018F939F930E94E725BF9193
:1052C000AF91A29F800D911DA39F900DB29F900D55
:1052D00011240895AA1BBB1B51E107C0AA1FBB1FC5
:1052E000A617B70710F0A61BB70B881F991F5A9572
:1052F000A9F780959095BC01CD01089597FB072EE5
:1053000016F4009407D077FD09D00E946A2907FCA3
:1053100005D03EF4909581959F4F089570956195C5
:105320007F4F0895DF93CF931F930F939A9DF02D96
:10533000219FF00D8B9DF00D8A9DE02DF10D039FB7
:10534000F00D029FE00DF11D4E9DE00DF11D5E9DE3
:10535000F00D4F9DF00D7F936F93BF92AF925F93CF
:105360004F93D5010E9453268B01AC01D7010E94B7
:105370005326EB01E80FF91FD6010E94E1292F9176
:105380003F91D6010E945326C60FD71FE81FF91F71
:10539000AF91BF910E94E1292F913F910E94532626
:1053A000C60FD71FE81FF91FD6010E945326E60F2C
:1053B000F71F9801BE01CF010F911F91CF91DF918F
:1053C00008950E945326460F571FC81FD91F08F47F
:1053D00031960895689401C0E894F92FF12B12F0EA
:1053E0000C941E2AA0E0B0E0E8EFF9E20C9400264D
:1053F000092E059422F40E947A2A112392F4F0E8EF
:105400000F26FFEFE094F09400951095B094C094AF
:10541000D094A194BF0ACF0ADF0AEF0AFF0A0F0B4C
:105420001F0B0E94292A07FC0E947A2ACDB7DEB7FB
:10543000ECE00C941C26689401C0E8948F929F9233
:10544000CF93DF930E94292ADF91CF919F908F9075
:10545000089588249924F401E401B0E49F93AA27D5
:105460009A158B049C04ED05FE05CF05D007A10716
:1054700098F4AD2FDC2FCF2FFE2FE92D982C892EFD
:10548000982F872F762F652F542F432F322F2227C7
:10549000B85031F7BF9127C01B2EBF91BB27220FF9
:1054A000331F441F551F661F771F881F991F881CB5
:1054B000991CEE1FFF1FCC1FDD1FAA1FBB1F8A14E4
:1054C0009B04EC05FD05CE05DF05A007B10748F0FC
:1054D0008A189B08EC09FD09CE09DF09A00BB10B66
:1054E00021601A94E1F62EF49401AF01BE01CD01C2
:1054F000000C089560957095809590953095409535
:10550000509521953F4F4F4F5F4F6F4F7F4F8F4FBC
:105510009F4F0895002E083090F0982F872F762FF8
:10552000652F542F432F322F22270850F4CF220FFC
:10553000331F441F551F661F771F881F991F0A9529
:10554000B2F7002D089597FD1094002E083098F0C2
:105550000850232F342F452F562F672F782F892F50
:10556000912DF4CF159497958795779567955795D5
:105570004795379527950A95AAF71124002D089588
:105580002A0D3B1D4C1D5D1D6E1D7F1D801F911F33
:1055900008952A193B094C095D096E097F09800BA2
:1055A000910B08950024A7FD00942A1730054005AB
:1055B000500560057005800590050895EE0FFF1FEA
:1055C0000590F491E02D09940F931F93CF93DF93EF
:1055D0008230910510F482E090E0E0916904F0914E
:1055E0006A0430E020E0B0E0A0E0309799F42115A3
:1055F000310509F44AC0281B390B24303105D8F590
:105600008A819B816115710589F1FB0193838283F6
:10561000FE0111C040815181028113814817590751
:10562000E0F04817590799F4109761F012960C931F
:10563000129713961C933296CF01DF91CF911F9151
:105640000F9108950093690410936A04F4CF211513
:10565000310551F04217530738F0A901DB019A01D7
:10566000BD01DF01F801C1CFEF01F9CF90936A04CA
:1056700080936904CDCFFE01E20FF31F81939193D4
:105680002250310939832883D7CF20916704309184
:105690006804232B41F420911001309111013093C3
:1056A00068042093670420910E0130910F012115A9
:1056B000310541F42DB73EB74091120150911301CD
:1056C000241B350BE0916704F0916804E217F3079F
:1056D000A0F42E1B3F0B2817390778F0AC014E5F62
:1056E0005F4F2417350748F04E0F5F1F5093680433
:1056F00040936704819391939FCFF0E0E0E09CCFCB
:10570000CF93DF930097E9F0FC0132971382128266
:10571000A0916904B0916A04ED0130E020E0109797
:10572000A1F420813181820F931F20916704309171
:1057300068042817390709F061C0F0936804E09302
:105740006704DF91CF910895EA01CE17DF07E8F5EE
:105750004A815B819E0141155105B1F7E901FB8347
:10576000EA8349915991C40FD51FEC17FD0761F4E5
:10577000808191810296840F951FE9019983888326
:10578000828193819B838A83F0E0E0E012968D9181
:105790009C9113970097B9F52D913C911197CD01EC
:1057A0000296820F931F2091670430916804281796
:1057B000390739F6309751F510926A04109269044E
:1057C000B0936804A0936704BCCFD383C2834081A5
:1057D0005181840F951FC817D90761F44E5F5F4F41
:1057E00088819981480F591F518340838A819B8109
:1057F000938382832115310509F0B0CFF0936A04B9
:10580000E09369049ECFFD01DC01C0CF13821282B8
:10581000D7CFB0E0A0E0EFE0FCE20C94FC258C01D7
:10582000009751F4CB010E94E42A8C01C801CDB746
:10583000DEB7E0E10C941826FC01E60FF71F9C018F
:1058400022503109E217F30708F49DC0D901CD9128
:10585000DC911197C617D70798F0C530D10530F302
:10586000CE0104978617970708F3C61BD70B22971C
:10587000C193D1936D937C93CF010E94802BD6CF9F
:105880005B01AC1ABD0A4C018C0E9D1EA0916904EF
:10589000B0916A04512C412CF12CE12C109731F578
:1058A00080916704909168048815990509F05CC09F
:1058B0004616570608F058C080910E0190910F01CE
:1058C000009741F48DB79EB740911201509113019A
:1058D000841B950BE817F90708F055C0F09368048E
:1058E000E0936704F90171836083A0CF8D919C914F
:1058F000119712966C90129713967C901397A81597
:10590000B90559F56C0142E0C40ED11CCA14DB0480
:1059100020F1AC014A195B09DA011296159780F063
:105920006282738251834083D9016D937C93E11429
:10593000F10471F0D7011396FC93EE93129776CF92
:1059400022968C0F9D1FF90191838083F301EFCF85
:10595000F0936A04E093690469CF4816590608F485
:105960002C017D01D3019ACFCB010E94E42A7C0156
:10597000009749F0AE01B8010E94CE2CC8010E94E8
:10598000802B870153CF10E000E050CF9111089594
:1059900081568A5108F4805285580895FB01DC0134
:1059A00002C001900D9241505040D8F70895FB017C
:1059B000DC0101900D920020E1F70895FB01DC016C
:1059C0004150504030F08D910190801919F4002021
:1059D000B9F7881B990B0895FB01DC014150504039
:1059E00048F001900D920020C9F701C01D9241506E
:1059F0005040E0F7089511E0C4ECD1E004C0FE018E
:105A00000E94DE2A2196C53CD107C9F7F894FFCF42
:105A10000101640016000000A0400000F0410000F9
:105A20006B04800000000000AB02F2013802F802B3
:105A3000690247025B02000000009E087108CD0861
:105A400037056A0857084808000000003805F201C9
:105A5000CD0837059405AC051F050D0A00543D001F
:105A60006F432000483D0025006F4320413D006DFD
:105A70000055563D00206E672F4C004C3D00424EB5
:105A80004D4C3033004E616E6F42326432504D00E7
:105A900073657269616C3A20002D35002D34002D3C
:105AA00033002D32002D3100440056657273696F4A
:105AB0006E3A200023007300534C20503D0050618B
:105AC00020697320756E6C696B656C792100536574
:105AD00061206C6576656C20503D00206850610047
:085AE00055565A005620000043
:107E0000112484B714BE81FFF0D085E080938100F7
:107E100082E08093C00088E18093C10086E0809377
:107E2000C20080E18093C4008EE0C9D0259A86E02C
:107E300020E33CEF91E0309385002093840096BBD3
:107E4000B09BFECF1D9AA8958150A9F7CC24DD24C4
:107E500088248394B5E0AB2EA1E19A2EF3E0BF2EE7
:107E6000A2D0813461F49FD0082FAFD0023811F036
:107E7000013811F484E001C083E08DD089C08234E0
:107E800011F484E103C0853419F485E0A6D080C0E4
:107E9000853579F488D0E82EFF2485D0082F10E0AE
:107EA000102F00270E291F29000F111F8ED06801E7
:107EB0006FC0863521F484E090D080E0DECF843638
:107EC00009F040C070D06FD0082F6DD080E0C81688
:107ED00080E7D80618F4F601B7BEE895C0E0D1E017
:107EE00062D089930C17E1F7F0E0CF16F0E7DF06D8
:107EF00018F0F601B7BEE89568D007B600FCFDCFD4
:107F0000A601A0E0B1E02C9130E011968C91119780
:107F100090E0982F8827822B932B1296FA010C0160
:107F200087BEE89511244E5F5F4FF1E0A038BF0790
:107F300051F7F601A7BEE89507B600FCFDCF97BE46
:107F4000E89526C08437B1F42ED02DD0F82E2BD052
:107F50003CD0F601EF2C8F010F5F1F4F84911BD097
:107F6000EA94F801C1F70894C11CD11CFA94CF0C13
:107F7000D11C0EC0853739F428D08EE10CD085E9AC
:107F80000AD08FE07ACF813511F488E018D01DD067
:107F900080E101D065CF982F8091C00085FFFCCF94
:107FA0009093C60008958091C00087FFFCCF809118
:107FB000C00084FD01C0A8958091C6000895E0E648
:107FC000F0E098E1908380830895EDDF803219F02E
:107FD00088E0F5DFFFCF84E1DECF1F93182FE3DFCA
:107FE0001150E9F7F2DF1F91089580E0E8DFEE27F6
:047FF000FF270994CA
:027FFE00040479
:00000001FF
